:020000040000FA
:0600000000000EEF00F00D
:0400080004EF00F011
:080018000CEF00F006D83FD9FF
:1000200014D96CD9CED877D8FAD78E0EC16EE10E1E
:10003000926EDC0E936ED80E946E0F0E956E000EBF
:10004000966E880ED56E100E806E20D801D81200E4
:10005000180EC86E280EC66E020E0E6E800E0B6E47
:10006000270E0D6E0F6A106A0B80900E056E020E41
:10007000066E00EE07F0AC0EEE6E0A0EED6E8FD837
:100080000B90900E056EEE0E8AD812000A0E036ECB
:1000900042D80306FDE18490050EF76ED20EF66E8F
:1000A00008008482F5CF83FF849235D88482F538A6
:1000B000836E849230D80B00F552F3E1050EF76E93
:1000C000DA0EF66E02D827D8120084900800F55296
:1000D00001E10B008482F5CF83FF84928482F5389E
:1000E000836E849213D884800B00F552F3E11200E2
:1000F00084908482EFCF83FF84928482EF38836E72
:10010000849204D88480EC50F4E11200210E036E36
:100110000306FEE11200F2A4FED7F2CF02F0F29E37
:10012000D6CF00F0D7CF01F0660E00269E0E01223A
:1001300001C0D7FF00C0D6FF0250800BF212F2942C
:1001400012000B849E96C5809EA6FED79E9605C083
:10015000C9FF9EA6FED79E96C5BC02D00B9401D0C7
:1001600001D81200050EF76EDC0EF66EAEDF050E3E
:10017000F76EE60EF66EA9DFBCEF00F012009E9659
:10018000C5829EA6FED79E9605C0C9FF9EA6FED735
:100190009E961200C5849EA6FED79E9612000590DC
:1001A000D0DF0BA008D0EECFC9FF9EA6FED79E964B
:1001B0000606F9E104D0C96E9EA6FED79E96EADF38
:1001C0001200090E0F26100E1026580E056E0B8019
:1001D000040E066E00EE0AF010C0EDFF010EED6E8B
:1001E0000FC0EDFFEF6ADBDF12000BA20BD0059012
:1001F000A8DF0BB406D0C96E9EA6FED79E960580DA
:10020000BEDF02D005809DDF0BB418D00BA00FD04D
:1002100017D8C9CFEEFF060602E0C59A01D0C58AFD
:10022000C5889EA6FED79E960650F2E107D008D854
:10023000C950C58AC5889EA6FED79E96ABDF120020
:10024000C5869EA6FED79E9612000C061DE1FA0EEC
:100250000C6E0EA213D00EA00BD00B90700E056E7C
:10026000FE0E9DDF0B90720E056EFE0E98DF05D020
:100270000B90700E056EFE0E92DF05D00B90720E85
:10028000056EFE0E8CDF0AD00B90700E056EFF0E11
:1002900086DF0B90720E056EFF0E81DF12000B9051
:1002A0000B92700E056EA1DF0BB40FD0800A800B8D
:1002B0000AE00B18800B06E180980B9E0E0602E107
:1002C000030E0E6E02D00B8E80881200046E036E39
:1002D0000A0E256EC3EC02F02050300FED6E0306BF
:1002E000F7E11C50300FEF6EEF50300A03E1200EA3
:1002F000EE6E01D0EE500406F7E112000D0621E18A
:10030000640E0D6E0B900B82900E056EAA0E6DDFC3
:100310000BB417D01C6E00EE16F0020ED7DF00EE05
:100320001AF0ED6A430EED6EDF0EED6E200EED6EEF
:1003300000EE13F0200EED6E200EED6E800EEF6ECF
:10034000D7DE120000000100018056550140343311
:10035000AB2A93240120721C9A1946175615B21322
:100360004A1212110110100F390E7A0DCD0C310CFA
:10037000A30B220BAB0A3E0AD9097C092509D40834
:10038000890843080108C207880751071D07EC06C2
:10039000BD06910667063F061906F505D205B105AB
:1003A0009105730556053A051F050605ED04D504AC
:1003B000BE04A80493047E046A045704450433046D
:1003C000220411040104F103E103D303C403B603BF
:1003D000A9039C038F03820376036A035F0354031C
:1003E00049033E0334032A03200316030D030403C9
:1003F000FB02F202E902E102D902D102C902C10202
:10040000BA02B202AB02A4029D02960290028902D5
:1004100083027D02770271026B0265025F025A025B
:1004200054024F024A0244023F023A0235023102AC
:100430002C02270223021E021A02150211020D02CB
:10044000090205020102FD01F901F501F101ED01C9
:10045000EA01E601E201DF01DB01D801D501D101AA
:10046000CE01CB01C801C401C101BE01BB01B8016D
:10047000B501B301B001AD01AA01A701A501A20117
:100480009F019D019A0198019501930190018E01B0
:100490008B01890187018401820180017E017B013A
:1004A000790177017501730171016F016D016B01B4
:1004B000690167016501630161015F015D015B0124
:1004C0005901580156015401520151014F014D018A
:1004D0004B014A01480147014501430142014001E6
:1004E0003F013D013C013A01390137013601340138
:1004F0003301310130012F012D012C012A01290185
:1005000028012601250124012201210120011F01CA
:100510001D011C011B011A0119011701160115010A
:1005200014011301120110010F010E010D010C0144
:100530000B010A0109010801070106010501040177
:10054000030102010101100E256008D025B6100C30
:1005500025B4200C25B2400C25B0800C25BC020C23
:1005600025BA040C25B8080C1FC023F01F6A1EC052
:1005700022F01E6A1DC021F01D6A1CC020F01C6AFA
:10058000000C206A000C010E2564C1EF02F01CC0B3
:1005900020F025501C6002D01C6A000CD890F76A2D
:1005A000E836F736450FF66E030EF7220A00F550CF
:1005B0002002F4CF1CF0F3CF1DF00800F55020020C
:1005C000F4501D26E86A1C2225501C02F350205EC0
:1005D000000C333228010C06000001008020446525
:1005E000766963652000C0204572726F722020001A
:020000040030CA
:08000000FFFAF6FEFFFFFBFF13
:00000001FF
